:030000000234FEC9
:0C34FE0078FFE4F6D8FD75814C023545DE
:1013A10020000A3C2E2E2E3E004950436F6E6E6582
:1013B10063745245510A004950436F6E6E65637400
:1013C100000A49504E6F41434B210A003E432C56BF
:1013D1002C43432CC0E4E0EFF2E5F020D1E8EDEA44
:1013E100EEEC49500A003E432C4D41432C2530324E
:1013F10062583A25303262583A25303262583A25DD
:10140100303262583A25303262583A2530326258C9
:101411002C4D414320E0E4F0E5F10A003E432C5617
:1014210045522C20332E3220EEF2202573202573D5
:101431002CC2E5F0F1E8FF20495020ECEEE4F3EB9B
:10144100FF0A004A756E20323520323030390031C2
:10145100343A30303A3131003E432C4C442C505216
:101461004F473A202020202020202020202020200B
:10147100202020202020202020202020202020206B
:10148100202020202020202020202020202020205B
:10149100202020202020202020202020202020204B
:1014A10020202020202020202CC4E0F2E020EFF09A
:1014B100EEF8E8E2EAE828F4E0E9EB290A003E2A3E
:1014C1002C312CCEF1EDEEE2EDFBE520EFE0F0E08A
:1014D100ECE5F2F0FB20F1E5F2E5E2EEE3EE20E8E7
:1014E100EDF2E5F0F4E5E9F1E00A003E412C41308E
:1014F100312C2562752E2562752E2562752E256289
:10150100752C495020E0E4F0E5F120E0E4E0EFF251
:10151100E5F0E00A003E412C4130322C2562752E67
:101521002562752E2562752E2562752C495020E0A5
:10153100E4F0E5F120EEF1ED2E20F1E5F0E2E5F049
:10154100E00A003E412C4130332C2562752E256284
:10155100752E2562752E2562752C495020E0E4F028
:10156100E5F120F0E5E72E20F1E5F0E2E5F0E00A13
:10157100003E412C4130342C2562752E2562752E9A
:101581002562752E2562752CCCE0F1EAE020F1E5AB
:10159100F2E80A003E412C4130352C2562752E259A
:1015A10062752E2562752E2562752CD8EBFEE70A31
:1015B100003E2A2C312CC4EEEF2E20EFE0F0E0ECBF
:1015C100E5F2F0FB20F1E5F2E5E2EEE3EE20E8EDF5
:1015D100F2E5F0F4E5E9F1E00A003E422C53303146
:1015E1002C2562752CC6E4E0F2FC20E7E0EFF0EE7A
:1015F100F1E020F1EEE5E4E8EDE5EDE8FF20EEF2C3
:1016010020F1E5F0E2E5F0E00A003E422C533032F1
:101611002C2562752CCEE1ECE5ED20F120F1E5F011
:10162100E2E5F0EEEC20E1E5E720EAE2E8F2E0EDC8
:10163100F6E8E90A003E422C5330332C2562752C22
:10164100CFE5F0E5E7E0EFF3F1EA20EFF0E820EF96
:10165100EEF2E5F0E520F1E2FFE7E820F120F1E527
:10166100F0E2E5F0EEEC0A003E454E440A000A4481
:10167100756D7058202020202030302030312030EE
:10168100322030332030342030352030362030378E
:101691002030382030392030412030422030432062
:1016A1003044203045203046000A3A003A20000AF2
:1016B100000A44756D7044202020202030302030F5
:1016C1003120303220303320303420303520303654
:1016D100203037203038203039203041203042202E
:1016E100304320304420304520304600457272207E
:1016F1006B657900526420656570726F6D0A0052E6
:1017010064204D454D0A00526420436F64650A0010
:10171100577269746520436F64650A004465627598
:10172100674950204F4E0A00446562756749502051
:101731004F46460A00446562756755736572204FCE
:101741006E0A00446562756755736572204F46469F
:101751000A0044656275674D7367204F6E0A004445
:10176100656275674D7367204F46460A00436F6E89
:10177100666967206C6F636B210A0057722065658B
:1017810070726F6D0A002053617665206565707215
:101791006F6D210A00457272204D414321004C6F4B
:1017A10061643E3E002A003C4130313D003C413005
:1017B100323D003C4130333D003C4130343D003C42
:1017C1004130353D003C21003C5330313D003C531C
:1017D10030323D003C5330333D003C5330353D0009
:0617E1003C5330363D00D0
:063D49000114000112004C
:103DA700C28E438910E4F58B758DB8D2ABD28E22C3
:03001B0002346E3E
:10346E00C0E0C083C082C0D0C28E758B00758DB88F
:10347E00201D0675A61E75A6E10512D219E514606B
:10348E00020514E513D39401400215130517E51731
:10349E00540F7048D225E517543F7012D21790661C
:1034AE008BE0600A04F0E0D394B44002D21D906623
:1034BE0086E0600204F0906104E0600214F0906611
:1034CE008CE0D394014003E014F0301C020515E5A6
:1034DE0016D394644004D21D80020516E511D394D0
:1034EE000140021511D28ED0D0D082D083D0E032DE
:10086900C291C290D2B5C2227D027C007F07123D9F
:100879002C8F26E526646060097D017F60123CC7E4
:10088900D222E4FDFC7F0B123D2C8F26E52630E6B3
:10089900097D04E4FF123CEBD2227D017C007F0735
:1008A900123D2C8F26E5267008FD7FFF123CC7D22A
:1008B90022302203126000C288C2A8C2AA75890028
:1008C90012382690633EE0B4FA06A3E064CE607B5A
:1008D900E4F52674362526F582E43463F583E4F0DD
:1008E9000526E526B443EC90633E74FAF0A374CE72
:1008F900F0A374CCF0906344740AF0E4A3F0A30469
:10090900F0A3F090633A74FFF0A3F0A3F0E4A3F02E
:10091900906355740AF0E4F526E5262401FFE433D3
:10092900FE74362526F582E43463F583E0FD123C36
:10093900A30526E526C3944340DFE4F5A775A61E63
:1009490075A6E1907FF0F0A3F080FE9063497403EF
:10095900F0A374CCF0E4906348F0123196C2B5125A
:1009690033CCC21D123AA8D222C224C22390657682
:100979007408F09062B47424F0E4A3F090633EE04C
:100989009062B6F090633FE09062B7F0906340E008
:100999009062B8F0906341E09062B9F0906342E0F0
:1009A9009062BAF0906343E09062BBF0751301E482
:1009B900906577F0C21EC21FC220C221202218AF43
:1009C90026FE7D03122E32E4FF12331C7E137FA113
:1009D900E4FBFDFC12285890668BE060037401F07B
:1009E900E4906104F0F515906575F0F516123DA7D0
:1009F90075A70775A61E75A6E1D2AFE4F516906135
:100A090004E07003122B5F90668CE06401701D9006
:100A190080007410F09080A874FFF0A3F0A3F0A3F5
:100A2900F0E490668CF0D222C223C224908008E0C0
:100A3900F52630E405D21E7410F0E52630E508D21B
:100A4900209080087420F0E52630E608D21F9080B7
:100A5900087440F0E515C394034019908002E4F04E
:100A6900908001F0908000F0E51594064006E4F5C9
:100A790015123AA89080A0E0700312391E9080B830
:100A8900E070031238A49080D0E07003123A4C90C1
:100A99008000E07013301E1012295F906331EFF06F
:100AA900D394004003120026908002E070069080E3
:100AB90000E06005D21C020A04C21CE4F51590612D
:100AC90004E06003020A04202212906578E0600CB9
:100AD9007E137FA3122D4AE4906578F0302012121C
:100AE9002464906331EFF0D394004005E0FF1200D5
:100AF9001F201F03020C7A1222DD906331EFF07080
:100B090003020A04906375E054BF247F7003020B4B
:100B1900E3147003020BBB24026003020C1C2022A5
:100B2900077E137FAA122D4A202603020C7A9063AE
:100B39004DE07006906351E06067906682E0FF9037
:100B4900634DE0B50724906683E0FE90634EE0B5FF
:100B59000618906684E0FE90634FE0B5060C906637
:100B690085E0FE906350E06E6037906351E06F60FE
:100B790003020C7A906683E0FF906352E06F600392
:100B8900020C7A906684E0FF906353E06F60030281
:100B99000C7A906685E0FF906354E06F6003020C65
:100BA9007AC21A9065777401F01200217513010257
:100BB9000C7A90668BE060037401F090667AE0FF2E
:100BC900906377E06F6003020C7A90667AE004F034
:100BD900E4F513906575F0020C7A301A03020C7A69
:100BE900906344E07003020A04906355740AF0129A
:100BF9000020D21AE4F513906575F090668604F02A
:100C0900E4906679F0A3F02022677E137FB8122D55
:100C19004A805E90668BE060037401F0301A52904E
:100C29006375E020E74B906377E0FF906679E0FE1B
:100C39006F600D906681E07007EE146F703380135A
:100C4900906679E004F0906331E0FFD394044003A7
:100C5900123B029060007482F0A37401F0906377F4
:100C6900E0906002F07E607F007D03123611020A77
:100C790004201A03020D92E5137068122141EF60F6
:100C8900237E647F75906476E02404FD123611900A
:100C99006681E07009906355E0F513020A04E4F5F2
:100CA90013020A04906686E0D3943C40369066812C
:100CB900E0703090668604F0123260E4906475F05A
:100CC900A37412F090667AE0906477F0A374FDF053
:100CD90090610563A20190647963A2017F12121EDB
:100CE9008F809E123D938F26E526B40115906000F2
:100CF9007483F0E4A3F07E607F007D021236110256
:100D09000A04E526D39401401C9060007483F0A383
:100D19007401F0E52624FEA3F07E607F007D0312B6
:100D29003611020A04E51364016003020A0490659E
:100D390075E004F02022077E137FC2122D4A9063CA
:100D490055E0C394C85004E02432F0906575E0C3BF
:100D59009405400DC21AE4906577F0120021020A49
:100D6900047C667D82906349E0FAA3E0FB7F02126E
:100D790037A27E647F75906476E02404FD123611F3
:100D8900906355E0F513020A04E513640160030258
:100D99000A04906577E014604624FE6042147003EB
:100DA900020E8524046003020A04E4F515202613C3
:100DB9009065777404F0906575E05401F07513013E
:100DC900020A049080027410F0E4906577F090654F
:100DD9007504F07513FA90668274FFF0020A0490A4
:100DE9006682E07003020E6F9064757480F09064FF
:100DF900777401F0E4A3F0A304F0A37430F0A374B2
:100E09007BF0E4F526747C2526F582E43464F583C9
:100E1900747DF0747D2526F582E43464F583E4F06D
:100E2900E5262407906476F07C667D82906349E02C
:100E3900FAA3E0FB7F021237A27E647F75E52624C0
:100E490009FD123611906681E0601B120020D21A4A
:100E5900E4F513906575F090668604F0E490667980
:100E6900F0A3F0020A04302607E4906577F08006C3
:100E79009065777404F07513FA020A04908002747D
:100E890010F0751305906575E06401FFF0906577C2
:100E99007401F0EF7019906351E06013FCA3E0FD59
:100EA900A3E0FEA3E0FF906682121C5B020A049095
:100EB900634DE0FCA3E0FDA3E0FEA3E0FF906682A2
:080EC900121C5B020A0480FE0A
:010ED10022FE
:10002600906376E0B444047F0180027F009063759C
:10003600E0B447047E0180027E00EE5F604A906372
:100046003EE0906377F090633FE0906378F09063D2
:1000560040E0906379F0906341E090637AF09063BA
:1000660042E090637BF0906343E090637CF09063A2
:10007600767452F09062AE63A2019080A863A201EA
:100086007F06121E8F02085F906331E0C39408500A
:100096000302086890633EE0FF906377E06F6003B9
:1000A60002086890633FE0FF906378E06F600302A8
:1000B6000868906340E0FF906379E06F6003020890
:1000C60068906341E0FF90637AE06F60030208681E
:1000D600906342E0FF90637BE06F600302086890E4
:1000E6006343E0FF90637CE06F60030208689063FF
:1000F60076E06444701A9080A8E0B4FF139062AE74
:1001060063A2019080A863A2017F06121E8F801051
:100116009062B2E09080ACF09062B3E09080ADF077
:1001260090668BE060037401F090668C7464F090C6
:1001360063767452F0906375E0646D600302026941
:100146007BFF7A1379CD1218497BFF7A1379E790F2
:10015600633EE0F52FA3E0F530A3E0F531A3E0F52B
:1001660032A3E0F533A3E0F534121849752FFF7575
:1001760030147531447532FF7533147534507BFF76
:100186007A14791D1218497BFF7A14795912184985
:100196007BFF7A1479BF1218497BFF7A1479EC90A9
:1001A6006344E0F52FA3E0F530A3E0F531A3E0F5D5
:1001B600321218497BFF7A15791690634DE0F52FB8
:1001C600A3E0F530A3E0F531A3E0F5321218497B40
:1001D600FF7A157944906351E0F52FA3E0F530A33B
:1001E600E0F531A3E0F5321218497BFF7A157972F2
:1001F60090633AE0F52FA3E0F530A3E0F531A3E0F4
:10020600F5321218497BFF7A157995906336E0F539
:100216002FA3E0F530A3E0F531A3E0F5321218493B
:100226007BFF7A1579B21218497BFF7A1579DBA222
:1002360026E433F52F1218497BFF7A16790B906660
:1002460081E0F52F1218497BFF7A16793690668B76
:10025600E0F52F1218491230CA7BFF7A1679691217
:10026600184922906375E0644C70737E167F6FFBAD
:10027600FDFC12285890637DE0F527A3E0F528E4FD
:10028600F52AE52790637FF0A3E528F07E167FAA7E
:100296007C637D7F7B02122858E4F52985288285B8
:1002A6002783E0FF747F2529F582E43463F583EF25
:1002B600F00528E528700205270529E529B410DC94
:1002C6007E167FAD7C637D7F7B10122858052AE55C
:1002D6002AC3941040AC7E167FB0122D4A2290633A
:1002E60075E0646C7060F52B7E167FB2FBFDFC1228
:1002F6002858E4F52AE490637FF0A3E52BF07E16F8
:100306007FAA7C637D7F7B02122858E4F529A82BFF
:10031600E6FF747F2529F582E43463F583EFF00563
:100326002B0529E529B410E67E167FAD7C637D7F1B
:100336007B10122858052AE52AC3940840B77E1672
:100346007FB0122D4A22906375E0644B7061F529E7
:1003560074672529F582E43463F583E060327467B7
:100366002529F582E43463F583E0F4602374672578
:1003760029F582E43463F583E0FF747D2529F5824F
:10038600E43463F583E0B507100529E529B408C010
:100396009061047432F002085F9063757421F03046
:1003A600220302085F7E167FED122D4A02085F9037
:1003B6006375E0B4521A2022077E167FF5122D4A85
:1003C6009063757472F07E637F757D0812358A229C
:1003D600906375E0644970452022077E177F0012FE
:1003E6002D4A90637DE0F527A3E0F528E4F52985FD
:1003F6002882852783E0FF747F2529F582E434630C
:10040600F583EFF00528E528700205270529E5297B
:10041600B480DC7E637F757D8A12358A229063758F
:10042600E0644370462022077E177F08122D4A900B
:10043600637DE0F527A3E0F528E4F5298528828584
:100446002783E493FF747F2529F582E43463F583DB
:10045600EFF00528E528700205270529E529B4806F
:10046600DB7E637F757D8A12358A22906375E06430
:100476005A70532022077E177F11122D4A90637DF2
:10048600E0F527A3E0F5287C637D7F7B80AF28AE6F
:1004960027123C48E4F529852882852783E493FFC3
:1004A600747F2529F582E43463F583EFF00528E5AA
:1004B60028700205270529E529B480DB7E637F7550
:1004C6007D8A12358A22906375E0644460030205D2
:1004D6005D90637DE0FF6444700302085FEFB43112
:1004E6000CC2227E177F1D122D4A02085F90637D83
:1004F600E0B4300CD2227E177F29122D4A02085F03
:1005060090637DE0B4320CD2237E177F36122D4ADB
:1005160002085F90637DE0B4330CC2237E177F44EC
:10052600122D4A02085F90637DE0B4340CD2247E1B
:10053600177F53122D4A02085F90637DE0B4350C95
:10054600C2247E177F60122D4A02085F90637DE009
:10055600FF12001E02085F906104E070132022075C
:100566007E177F6E122D4A9063757421F002085F24
:100576009061047432F0906375E0FFB45104C2AF29
:1005860080FEEF645770452022077E177F7C122D70
:100596004A90637EE0906331F0E4F529906331E0A0
:1005A600FFE529C39F400302085F747F2529F58272
:1005B600E43463F583E0FF90637DE0252924ADF5FF
:1005C60082E43461F583EFF0052980D0906375E00D
:1005D600645360030206802022077E177F87122D50
:1005E6004A90633EE0FF9061B6E06F703C90633FD7
:1005F600E0FF9061B7E06F7030906340E0FF90617C
:10060600B8E0B50724906341E0FF9061B9E0B50713
:1006160018906342E0FF9061BAE0B5070C9063431F
:10062600E0FF9061BBE06F60169063757421F03057
:10063600220302085F7E177F96122D4A02085FE4A6
:10064600F529E4F516AF29FE74AD2529F582E434C3
:1006560061F583E0FD123CA30529E529C394FE401C
:10066600E1C2AFE4907FF0F0A3F0907FFD74AAF0B2
:10067600A374FFF0A37455F080FE906375E0644F99
:10068600704C90637DE0F527A3E0F528E528452723
:10069600700A2022077E177F9F122D4A2022077E8E
:1006A600177FA6122D4AE4F529747F2529F582E4E1
:1006B6003463F583E0852882852783F00528E528BD
:1006C600700205270529E529B480DE02085F9063DC
:1006D60075E0FFB4452190637DE0FDA3E0907FF0D7
:1006E600CDF0A3EDF0C2AF907FFD74AAF0A374FF26
:1006F600F0A37455F080FEEF64656003020868900D
:10070600637DE0FFA3E0907FF0CFF0A3EFF0E4F588
:1007160027F528D3907FF1E09528907FF0E0952784
:100726004020E4F5162528FFE5273401FE852882BA
:10073600852783E0FD123CA30528E52870020527DE
:1007460080D17E177FA8123698EF4E6020120003E4
:10075600906344EFF0120003906345EFF01200033C
:10076600906346EFF0120003906347EFF07E177F29
:10077600AE123698EF4E602012000390634DEFF0F4
:1007860012000390634EEFF012000390634FEFF0F8
:10079600120003906350EFF07E177FB4123698EF85
:1007A6004E6020120003906351EFF0120003906335
:1007B60052EFF0120003906353EFF01200039063C0
:1007C60054EFF07E177FBA123698EF4E6020120073
:1007D6000390633AEFF012000390633BEFF01200D0
:1007E6000390633CEFF012000390633DEFF07E1739
:1007F6007FC0123698EF4E6020120003906336EFEA
:10080600F0120003906337EFF0120003906338EFA5
:10081600F0120003906339EFF0E4F529E4F516E5EC
:10082600292401FFE433FE74362529F582E4346376
:10083600F583E0FD123CA30529E529C3944340DC7A
:10084600C2AFE4907FF0F0A3F0907FFD74AAF0A30E
:1008560074FFF0A37455F080FE7E637F757D0812E9
:02086600358AD1
:01086800226D
:103BDB00AE07EEC39430400BEED394395005EE2470
:103BEB00D0FF22EEC39461400BEED394665005EEEA
:103BFB0024A9FF22EEC39441400BEED3944650050B
:083C0B00EE24C9FF22AF0622DE
:103D65009062ADE004F070069062ACE004F0906201
:0A3D7500ACE0FEA3E0FF123D0F22B8
:10000300123D65123BDBEFC454F0FEC006123D65A2
:08001300123BDBD0E02FFF22BD
:1039EF00E4906AC2F0123D65906AC3EFF0C3943061
:1039FF004018E0FFD394395011906AC2E02405F5C6
:103A0F0082E43461F583EFF08011906AC2E02405FF
:103A1F00F582E43461F583E4F0800C906AC2E0042F
:103A2F00F0E0D3940840BE752A00752B00752C006A
:0C3A3F00E4F52D7B017A617905121F9DD2
:013A4B002258
:043698008E2C8F2DB8
:10369C009062ACE4F0A374FFF0123D65EF606EF441
:1036AC00606B852D82852C83E493B507EC752E0118
:1036BC00E52D252EF582E4352CF583E493602590D9
:1036CC0062ADE0252EFF9062ACE03400FE123D0F9F
:1036DC00E52D252EF582E4352CF583E493B507040E
:1036EC00052E80CCE52D252EF582E4352CF583E4D2
:1036FC009370A6E52E24FFFFE434FFFE9062ADE04C
:10370C002FF09062ACE03EF07E007F0122E4FEFFE1
:01371C00228A
:103196007E177FC6123698EF4E70037F01227E1788
:1031A6007FC9123698EF4E600C123D65EF24D0248D
:1031B600FF92268002D2267E177FCF123698EF4ED8
:1031C600600C123D65EF24D0906681F08005E49096
:1031D6006681F07E177FD5123698EF4E600C123D51
:1031E60065EF24D090668BF08005E490668BF07EC8
:1031F600177FDB123698EF4E600C123D65EF24D038
:1032060024FF92188002C21890633E63A201906662
:103216007B63A2017F06121E8F30183B7E177FE16B
:10322600123698EF4E603012000390667BEFF01274
:10323600000390667CEFF012000390667DEFF012BB
:10324600000390667EEFF012000390667FEFF012A7
:0A3256000003906680EFF07F002275
:103B5900906576E0C3947C40027F0A906576E0FE2A
:103B690004F074B42EF582E43462F583EFF0BF0AF1
:103B790027906576E0FF04F074B42FF582E434628F
:103B8900F583E4F0906576E0FF12371D9065767451
:093B990008F09062B5E004F0228E
:100ED2003E2A2C312CCFE0F0E0ECE5F2F0FB20E0F2
:100EE200F1E8EDF5F0EEEDEDEEE3EE20EFEEF0F2EF
:100EF200E02E20D0E5E6E8EC20F0E0E1EEF2FB2087
:100F02002D20EFE0EAE5F2EDFBE920EFEE2055447B
:100F12005020E820EAE2E0E7E8EFEEF2EEEAEEE265
:100F2200FBE920EFEE205443500A003E432C4B30A5
:100F3200362C25732CD2E5EAF3F9E8E920F0E5E650
:100F4200E8EC0A003E4C2C4930312C256C752CD132
:100F5200EAEEF0EEF1F2FC20EEE1ECE5EDE02C350C
:100F6200302C3130302C3330302C3630302C313282
:100F720030302C323430302C343830302C3936305A
:100F8200302C31393230302C33383430302C353744
:100F92003630302C3131353230300A003E422C4965
:100FA20030322C2562752CD3EFF0E0E2EBE5EDE870
:100FB200E520EFEEF2EEEAEEEC20EFF0E820EFE5CE
:100FC200F0E5E4E0F7E520285254532D4354532929
:100FD2000A003E532C4930332C2562752CC7E0E4BD
:100FE200E5F0E6EAE020F1F2E0F0F2E020EFE5F0F1
:100FF200E5E4E0F7E8282A3130ECF1290A003E4224
:101002002C4930342C2562752CD0E5E6E8EC20EF33
:10101200E5F0E5E4E0F7E8203720E1E8F20A003EF7
:10102200422C4930352C2562752CCFE5F0E5E4E001
:10103200F7E020F120EAEEEDF2F0EEEBFCEDFBEC56
:1010420020E1E8F2EEEC0A003E422C4930362C2533
:1010520062752CCAEEEDF2F0EEEBFCEDFBE920E15D
:10106200E8F2202D20F7E5F2EDEEF1F2FC0A003E67
:10107200422C415030372C2562752CC6E4E0F2FC3C
:1010820020EAE2E8F2E0EDF6E8FE20EEF220F3F1EB
:10109200F2F0EEE9F1F2E2E00A003E422C41503079
:1010A200382C2562752CCAE2E8F2E8F0EEE2E0F2B2
:1010B200FC20EFE0EAE5F2FB20EEF220F3F1F2F0A1
:1010C200EEE9F1F2E2E00A003C21003C4930313D18
:1010D200003C4930323D003C4930333D003C493010
:1010E200343D003C4930353D003C4930363D003C02
:1010F200415030373D003C415030383D000A536585
:101102006E64205061636B65743A20000A53656E09
:1011120064204B56543A20000AC1F3F4E5F020E76C
:10112200E0EDFFF221000A435243206572726F72B2
:1011320021202020000ACEF2E2E5F7E0FE20EDE0D9
:1011420020E7E0E3F0F3E7EAF321000A52656320C7
:101152004B5654000A526563206F6B2120202020D9
:10116200202000496E69745443500A004C6973741C
:10117200656E5443500A00534F434B5F5443505FD4
:1011820045535441424C49534845440A000A2D3EB6
:1011920020000A3C2D2000544350005544500000CA
:1011A200112332465765748C9DAFBECADBE9F81035
:1011B200013322564775649C8DBFAEDACBF9E82124
:1011C20030021367764455ADBC8E9FEBFAC8D93115
:1011D20020120377665445BDAC9E8FFBEAD8C94204
:1011E20053617004152736CEDFEDFC8899ABBA52F5
:1011F20043716014053726DECFFDEC9889BBAA63E4
:1012020072405125340617EFFECCDDA9B88A9B73D4
:1012120062504135241607FFEEDCCDB9A89A8B84C3
:1012220095A7B6C2D3E1F008192B3A4E5F6D7C94B4
:1012320085B7A6D2C3F1E018093B2A5E4F7D6CA5A3
:10124200B48697E3F2C0D129380A1B6F7E4C5DB594
:10125200A49687F3E2D0C139281A0B7F6E5C4DC683
:10126200D7E5F48091A3B24A5B69780C1D2F3ED674
:10127200C7F5E49081B3A25A4B79681C0D3F2EE763
:10128200F6C4D5A1B082936B7A48592D3C0E1FF754
:10129200E6D4C5B1A092837B6A58493D2C1E0F004B
:1012A20089129B24AD36BF48C15AD36CE57EF781C3
:1012B20008931AA52CB73EC940DB52ED64FF7602B3
:1012C2008B109926AF34BD4AC358D16EE77CF583A3
:1012D2000A9118A72EB53CCB42D950EF66FD740493
:1012E2008D169F20A932BB4CC55ED768E17AF38583
:1012F2000C971EA128B33ACD44DF56E960FB720673
:101302008F149D22AB30B94EC75CD56AE378F18762
:101312000E951CA32AB138CF46DD54EB62F9700852
:10132200811A932CA53EB740C952DB64ED76FF8942
:10133200009B12AD24BF36C148D35AE56CF77E0A32
:101342008318912EA73CB542CB50D966EF74FD8B22
:10135200029910AF26BD34C34AD158E76EF57C0C12
:10136200851E9728A13AB344CD56DF60E972FB8D02
:10137200049F16A920BB32C54CD75EE168F37A0EF2
:10138200871C952AA338B146CF54DD62EB70F98FE2
:0F139200069D14AB22B930C74ED55CE36AF178E3
:103D4F0052668D000000000000000000000000001F
:053D5F0000000000005F
:103C7C0074AE2548F582E43467F583EFF00548907F
:103C8C0067ACE548F064646005E548B4E408D20824
:073C9C0063488053488022B9
:01001E0022BF
:030023000227248D
:0B272400C0E0C083C082C0D075D01898
:10272F002098030227DA751401AE9920021ABE020F
:10273F0012D291300F05AF1E123C7C754505D202A7
:10274F000227D8C2910227D8300E1EC20E300F07B3
:10275F00AF1E123C7C806FAF48054874AE2FF582D8
:10276F00E43467F583EEF0805DBE090C300F05AFE2
:10277F001E123C7CD20E804EBE020D534880300F8D
:10278F0045AF1E123C7C803EEE6403701F300F0776
:10279F00AF1E123C7C80069067ACE548F063488022
:1027AF00534880C202D208754500801A300F07AF18
:1027BF001E123C7C8010AF48054874AE2FF582E4A2
:1027CF003467F583EEF0754505C298309970300384
:1027DF006B301007309704D20080619066A1E0FF44
:1027EF00E549C39F4011C203D213C290200B02D2FE
:1027FF0015C20BD2968045AF49054974AE2FF582AD
:10280F00E43468F583E0F54A300919534A7F300103
:10281F002820D008200422634A80801D30041A63C8
:10282F004A808015300112E54A524A300406A2D080
:10283F00929B8005A2D0B3929B854A99C299D2AF41
:09284F00D0D0D082D083D0E03259
:1030CA007BFF7A0E79D2121849300F14752FFF75CB
:1030DA0030117531997BFF7A0F792D1218498012B8
:1030EA00752FFF75301175319D7BFF7A0F792D127F
:1030FA0018499069AEE0FEA3E0FFC3E49FFFE49E97
:10310A00FEAB07FA3395E0F9F87F007E8C7D0A7CE6
:10311A0000121BAA8F328E318D308C2F7BFF7A0FD3
:10312A0079461218497BFF7A0F799EA210E433F58B
:10313A002F1218497BFF7A0F79D485462F12184926
:10314A007BFF7A107900A209E433F52F1218497B24
:10315A00FF7A107921A201E433F52F1218497BFF77
:10316A007A10794AA204E433F52F1218497BFF7AC0
:10317A00107971A211E433F52F1218497BFF7A10E6
:0C318A00799CA20AE433F52F12184922A8
:102A63007E107FCA123698EF4E70037F01227E10CC
:102A73007FCD123698EF4E60231239EFA804A905D3
:102A8300AA06AB077F007E8C7D0A7C00121BAA126C
:102A93001C3C9069AEEEF0A3EFF0800A9069AE742F
:102AA300FFF0A374B8F07E107FD3123698EF4E6018
:102AB3000C123D65EF24D024FF92108002C2107ED9
:102AC300107FD9123698EF4E60071239EF8F468088
:102AD30003E4F5467E107FDF123698EF4E600C124A
:102AE3003D65EF24D024FF92098002C2097E107F46
:102AF300E5123698EF4E600C123D65EF24D024FFAB
:102B030092018002C2017E107FEB123698EF4E6075
:102B13000C123D65EF24D024FF92048002C2047E90
:102B2300107FF1123698EF4E600E123D65EF24D000
:102B330024FF920592118004C205C2117E107FF812
:102B4300123698EF4E600E123D65EF24D024FF92AB
:0C2B530005920A8004C205C20A7F00221D
:1033CC00C203C215C208C202C20EE4F5499066A13E
:1033DC00F0F548F514C200D297D2969067ADF0C2C2
:1033EC0006C21490669F7409F0A3F0C209C204C20D
:1033FC0001C212C210E4F546F545D2139069AE74C1
:10340C00FFF0A374B8F0C20AC205C211122A63906D
:10341C0067A27401F0C2ADE4F5C9D2CDD2CCC2C959
:10342C00C2CAF5CDF5CC9069AEE0F5CBA3E0F5CAF8
:10343C0085CBCD85CACCE4F59830010C2009095315
:10344C0087BFD29FD29E8002D29E438740C29FC22A
:10345C00ACC298C29975B81075B710D2CAD29CD2AA
:02346C00AC2290
:103D7F00E54C6FFF9012A193654BF54CEF9011A19D
:033D8F0093F54B5E
:013D9200220E
:01001F0022BE
:0425D5008E288F2994
:1025D900E4F52AF54CF54BAA06A9077B018B2E8A4F
:1025E9002F8930121B5C042530F530E4352FF52F87
:1025F90030050F9067A3E0AB2EAA2FA930121B5C00
:10260900800D9066A0E0AB2EAA2FA930121B5C7535
:102619002E0185282F8529300D0DE4FEEEC39D502E
:1026290018AB2E0530E530AA2F7002052F14F912C8
:102639001B43FF123D7F0E80E3AB2E0530E530AA28
:102649002F7002052F14F9E54C121B5CAB2EAA2F33
:10265900A930E54B121B5C0D0D752C68752DAE75F7
:102669002E0185282F852930852D82852C8374029A
:10267900F0052DE52D7002052C052AE4FEEEC39D1B
:10268900504EAB2EAA2FA930121B43F52B640260C2
:102699000BE52B64036005E52BB40913852D8285B1
:1026A9002C837409F0052DE52D7002052C052A856A
:1026B9002D82852C83E52BF0052DE52D7002052C47
:1026C900052A74012530F530E4352FF52F0E80AD3C
:1026D900852D82852C837403F0052DE52D70020567
:1026E9002C052A906693E0FCA3E0FDA3E0FEA3E09D
:1026F900FFE4FAF9F8EF2401FFEA3EFEE93DFDE8BF
:102709003CFC906693121C5B30240D7E107FFF7C8D
:0A271900687DAEAB2A122858AF2AE3
:012723002293
:10326000E4FF9066A0E0FE7D000FED2405F582E40A
:103270003461F583EEF00F74052401F582E43461C6
:10328000F583E4F07C667D92FEED1DAA0470011CBE
:10329000F5828A83E0FBAA070F74052AF582E434DD
:1032A00061F583EBF00EBE04E07C667D96E4FEEDF6
:1032B0001DAA0470011CF5828A83E0FBAA070F7423
:1032C000052AF582E43461F583EBF00EBE04E07C60
:1032D000667D9AE4FEED1DAA0470011CF5828A83C6
:1032E000E0FBAA070F74052AF582E43461F583EB4D
:1032F000F00EBE04E07C667D9EE4FEED1DAA047027
:10330000011CF5828A83E0FBAA070F74052AF58267
:0B331000E43461F583EBF00EBE04E036
:01331B00228F
:0A3DC200C2992099FDD299D29022F7
:0100200022BD
:103BA200AD07200F337E677FA21225D59066A1EF65
:103BB200F0D203E4F54930240D7E117F0E7C687D3E
:103BC200AEE0FB122858C296301003D20022E5461E
:093BD2006003F51122123DC2222C
:103B02008F27200F5130030F30244B7E117F1AE490
:103B1200FBFDFC12285822906378E09066A0F07EAC
:103B2200637F77E52724FCFD1225D59066A1EFF08F
:103B3200A21182055005754705D214E4F549D20356
:103B4200C296301004D200800BE5466004F5118065
:073B520003123DC2C215225F
:10214100200603300B037F00222008030222D23035
:102151000F037F0022C208C291E4906475F090677A
:10216100ACE0FF547F24FCF527906476F090667A0A
:10217100E0906477F0EF5480FF24AFF582E4346798
:10218100F583E0906478F074AE2FF582E43467ADA6
:1021910082FCE4F54CF54BFE9067ACE0547FF9EE20
:1021A100C39950140DEDAA0470010C14F5828A83B1
:1021B100E0FF123D7F0E80E0E54B454C604430244A
:1021C100197E117F289067ACE0548024AEF582E43B
:1021D1003467AD82FCAB01122858906697E0FCA3EE
:1021E100E0FDA3E0FEA3E0FFE4FAF9F8EF2401FF2C
:1021F100EA3EFEE93DFDE83CFC906697121C5B025D
:1022010022D23005249067ACE05480FF24AEF582E1
:10221100E43467F583E09067A2F074AF2FF582E4B0
:102221003467F583E09067A3F0E5277039C214F5B0
:10223100479067A3E0B4E01E7490F02005030222EA
:10224100D2D2062024030222D27E117F37E4FBFD85
:10225100FC122858807B3024787E117F4DE4FBFDF1
:10226100FC122858806B9067ACE0548024B0F58252
:10227100E43467F58363A20190647963A201AF2717
:10228100121E8F30241C7E117F569067ACE0FB54E8
:102291008024AEF582E43467AD82FCEB547FFB12FF
:1022A100285890668FE0FCA3E0FDA3E0FEA3E0FFC9
:1022B100E4FAF9F8EF2401FFEA3EFEE93DFDE83CCE
:1022C100FC90668F121C5BA20A82055002D206D2D4
:0B22D10016301605C2167F01227F00A8
:0122DC0022DF
:103C130030082FC208C291300F289067ACE0FF54E0
:103C23008024AEF582E43467F58363A2019069B41E
:103C330063A201EF547FFF121E8F9067ACE0547FA5
:053C4300FF227F0022BA
:0100210022BC
:102B5F003017469080E8E0700F12398C3024077ED2
:102B6F00117F65122D4AC20F9080E8E0B40E1290CB
:102B7F0080037408F03024077E117F6E122D4AC235
:102B8F000F9080E8E0B4060F200F0C3024077E1161
:102B9F007F79122D4AD20FC217300F5E2003071212
:102BAF002F138F278003E4F527E527603130240C9E
:102BBF007E117F8F7C697DB4FB1228589069B463B6
:102BCF00A2019068AE63A201AF27121E8F9066A17B
:102BDF00E527F0E4F549D290D203C296D299123C80
:102BEF00138F27E5276013122C5A30240D7E117F87
:102BFF00947C697DB4AB27122858300008209705C4
:102C0F00C200123DC2E511B40106E4F511123DC236
:102C1F00302525C225E545600DD5450A634880530B
:102C2F004880C202C29130110FE547600BD54708AB
:102C3F00E4F549D203754705A20A8206500C20031A
:0A2C4F0009E4FF123BA2C206D20BFB
:012C59002258
:103D9300300F037F0022301508201405C2157F0160
:043DA300227F002259
:103AA8009080007480F090633663A201F583F582FC
:103AB80063A2017F08121E8F90633E63A20190806B
:103AC8008863A2017F0A121E8F9080927407F0A368
:103AD80074D0F0A37406F0906348E0FF9080B1F0D2
:103AE8009080E1EFF09080957455F0A3F0908000FD
:0A3AF8007401F090800974F0F022D0
:10391E00908009E04410F09080A0E070609080A14B
:10392E007482F09080A874FFF0A3F0A3F0A3F07F50
:10393E00039080AEEFF0A374CBF09080007402F091
:10394E00906AB4121C6700000000906AB4E0908088
:10395E0040F0906AB5E0908041F0906AB6E09080B9
:10396E0042F0906AB7E0908043F0A3E4F0A3F0A396
:0D397E00F0A3F0908018F0A3F0A3F0A3F0E8
:01398B002219
:103A4C00908009E04440F09080D17482F07F039024
:103A5C0080DEEFF0A374CCF09080027402F0906AD8
:103A6C00B8121C6700000000906AB8E0908058F013
:103A7C00906AB9E0908059F0906ABAE090805AF060
:103A8C00906ABBE090805BF0A3E4F0A3F0A3F0A3FA
:0B3A9C00F0908030F0A3F0A3F0A3F046
:013AA70022FC
:1038A400908009E04420F09080B8E0706C9080B97A
:1038B4007482F07F039080C6EFF07FCDA3EFF07F9A
:1038C400039080C4EFF0A374CDF09080C074FFF037
:1038D400A3F0A3F0A3F09080017402F0906ABC12EC
:1038E4001C6700000000906ABCE090804CF0906A75
:1038F400BDE090804DF0906ABEE090804EF0906AFA
:10390400BFE090804FF0A3E4F0A3F0A3F0A3F09005
:093914008024F0A3F0A3F0A3F05D
:01391D002287
:1037A2008C278D28A907EAFDE975F018A424ACFF3F
:1037B200E5F034808F82F583EDF0EBFDE975F018CA
:1037C200A4FFAEF024ACFBEE34808B82F583A3ED34
:1037D200F08528828C83E0FDEF24A8FFEE3480FE82
:1037E2008F82F583EDF08528828C83A3E08F828E11
:1037F20083A3F0852882852783A3A3E0FDE975F0E2
:1038020018A424A8FFE5F03480FE8F82F583A3A3D9
:10381200EDF08528828C83A3A3A3E08F828E83A3FD
:04382200A3A3F0224A
:06358A008D2CAB07AA0620
:10359000908000E030E5079065787401F022906A31
:1035A000B4E0FCA3E0FDA3E0FEA3E0F5308E2F8D98
:1035B0002E8C2DAE02AF038E838F8263A201E52F86
:1035C000540744C0F58385308263A201AF2C121FDB
:1035D00001E4FCFDFEE530252CF530EE352FF52F0E
:1035E000ED352EF52EEC352DF52D908040E52DF0A6
:1035F000A3E52EF0A3E52FF0A3E530F09080007452
:1036000020F0AF30AE2FAD2EAC2D906AB4121C5B03
:013610002297
:063611008D27AB07AA069D
:10361700908002E030E5079065787403F022906AA5
:10362700B8E0FCA3E0FDA3E0FEA3E0F52B8E2A8D16
:10363700298C28AE02AF038E838F8263A201E52A0D
:10364700540744D0F583852B8263A201AF27121F4D
:1036570001E4FCFDFEE52B2527F52BEE352AF52A9F
:10366700ED3529F529EC3528F528908058E528F01F
:10367700A3E529F0A3E52AF0A3E52BF090800274D7
:1036870020F0AF2BAE2AAD29AC28906AB8121C5B8C
:013697002210
:02331C008F27F9
:10331E00908001E030E5099065787402F07F00221C
:10332E00906ABCE0FCA3E0FDA3E0FEA3E0F52B8ECB
:10333E002A8D298C2890667B63A201E52A540744C6
:10334E00C8F583852B8263A2017F06121F17E52B1A
:10335E002406F52BE4352AF52AE43529F529E4353A
:10336E0028F52890657963A201E52A540744C8F52B
:10337E0083852B8263A201AF27121F17E4FCFDFE8B
:10338E00E52B2527F52BEE352AF52AED3529F529DE
:10339E00EC3528F52890804CE528F0A3E529F0A31C
:1033AE00E52AF0A3E52BF09080017420F0AF2BAE50
:0D33BE002AAD29AC28906ABC121C5BAF2719
:0133CB0022DF
:10295F009081E0E0F527052705270527052705279F
:10296F0005270527052705270527908010E0F52A5D
:10297F00A3E0F52BA3E0F52CA3E0F52D9081E1E08A
:10298F00F5270527052705270527052705270527E8
:10299F00052705270527908014E0F52EA3E0F52FD6
:1029AF00A3E0F530A3E0F531E530B52C08E531B5FE
:1029BF002D037F0022E4F527E530540744E0F5832B
:1029CF0085318263A20190637563A2017F08121F94
:1029DF004790637763A2019062AE63A2017F0612F4
:1029EF001E8F906375E0F528A3E0F529E4F5279095
:1029FF006375E0702AA3E024F8F527E53054074407
:102A0F00E0F58385318274082582F582E43583F5FC
:102A1F008363A20190637563A201AF27121F47AEB4
:102A2F0028E4FCFDE5312529F531E5303EF530EDA3
:102A3F00352FF52FEC352EF52E908014E52EF0A3C3
:102A4F00E52FF0A3E530F0A3E531F090800074405E
:032A5F00F0AF27AE
:012A62002251
:1022DD009081E6E0F5270527052705270527052722
:1022ED0005270527052705270527908028E0F52ACE
:1022FD00A3E0F52BA3E0F52CA3E0F52D9081E7E00D
:10230D00F527052705270527052705270527052770
:10231D0005270527052790802CE0F52EA3E0F52F46
:10232D00A3E0F530A3E0F531E4F527E530B52C0A4F
:10233D00E531B52D05C21F022449E530540744F09F
:10234D00F58385318263A20190637563A2017F08D5
:10235D00121F47906375E0F528A3E0F529E529459F
:10236D002870099080027410F07F0022906682E040
:10237D00FFF46030906377E06F6003022410906685
:10238D0083E0FF906378E06F7079906684E0FF9052
:10239D006379E06F706D906685E0FF90637AE06F12
:1023AD006031805F906377E0906682F0906378E0B3
:1023BD00906683F0906379E0906684F090637AE0A4
:1023CD00906685F090637BE0FFA3E0906349CFF0CA
:1023DD00A3EFF0906375E0702AA3E024F8F527E5EC
:1023ED0030540744F0F58385318274082582F582D7
:1023FD00E43583F58363A20190637563A201AF2772
:10240D00121F47AE28E4FCFDE5312529F531E530F5
:10241D003EF530ED352FF52FEC352EF52EAF2DAEDB
:10242D002CAD2BAC2AAB31AA30A92FA82ED3121C60
:10243D004A40099080027410F07F002290802CE5B4
:10244D002EF0A3E52FF0A3E530F0A3E531F0908059
:06245D00027440F0AF27FD
:012463002256
:102464009081E3E0F527052705270527052705279C
:102474000527052705270527052790801CE0F52A51
:10248400A3E0F52BA3E0F52CA3E0F52D9081E4E087
:10249400F5270527052705270527052705270527E8
:1024A400052705270527908020E0F52EA3E0F52FCA
:1024B400A3E0F530A3E0F531E4F527E530B52C0AC7
:1024C400E531B52D05C2200225BAE530540744E8AC
:1024D400F58385318263A20190600463A2017F0EBB
:1024E400121F5D906004E0F528A3E0F52990600CCC
:1024F400E0FFF4604A90667BE0FEEF6E7079A3E043
:10250400FF90600DE06F706F90667DE0FF90600E4D
:10251400E06F706390667EE0FF90600FE06F70572D
:1025240090667FE0FF906010E06F704B906680E0F3
:10253400FF906011E06F703FE4906013F0800890AA
:10254400601374FFF0D2D9906004E0702AA3E024F1
:10255400F2F527E530540744E8F583853182740E9B
:102564002582F582E43583F58363A20190600463D8
:10257400A201AF27121F5DAE28E4FCFDE531252939
:10258400F531E5303EF530ED352FF52FEC352EF5F0
:102594002EAF2DAE2CAD2BAC2AAB31AA30A92FA86F
:1025A4002ED3121C4A5006E5294528700990800153
:1025B4007410F07F0022908020E52EF0A3E52FF028
:1025C400A3E530F0A3E531F09080017440F0AF272B
:0125D40022E4
:042D4A008E2C8F2D0F
:102D4E00908000E030E5079065787401F022906A7B
:102D5E00B4E0FCA3E0FDA3E0FEA3E0F5338E328DDC
:102D6E00318C30E533FFE5325407FEE42FF52FEEBC
:102D7E0034C0F52E852F82F5837423F0052FE52FB1
:102D8E007002052E532EC7F582852E83740AF00528
:102D9E002FE52F7002052E532EC790633E63A201BE
:102DAE00852E83852F8263A2017F06121F01740672
:102DBE00252FF52FE4352EF52E852C83852D826358
:102DCE00A201852E83852F8263A201121EE5E4FCEB
:102DDE00FDFE906AB4E0F8A3E0F9A3E0FAA3E02FB9
:102DEE00FFEE3AFEED39FDEC38FCEF2408FFE43E31
:102DFE00FEE43DFDE43CFC906AB4121C5B906AB4A8
:102E0E00E0908040F0906AB5E0908041F0906AB614
:102E1E00E0908042F0906AB7E0908043F09080009E
:032E2E007420F01D
:012E3100227E
:0A2858008E318F328C338D348B35B6
:10286200908000E030E5079065787401F022906A6C
:10287200B4E0FCA3E0FDA3E0FEA3E0F53B8E3A8DBD
:10288200398C38E53BFFE53A5407FEE42FF537EE85
:1028920034C0F536853782F5837423F00537E53782
:1028A200700205365336C7F582853683740AF00501
:1028B20037E537700205365336C790633E63A2018F
:1028C20085368385378263A2017F06121F01740653
:1028D2002537F537E43536F536853183853282631F
:1028E200A20185368385378263A201121EE58F3CE1
:1028F200EF2537F537E43536F536E535601785339C
:102902008385348263A20185368385378263A2017F
:10291200AF35121F01E53C24082535F535FFE4FCEF
:10292200FDFEE53B2FF53BEE353AF53AED3539F54F
:1029320039EC3538F538908040E538F0A3E539F0C8
:10294200A3E53AF0A3E53BF09080007420F0AF3BA2
:0C295200AE3AAD39AC38906AB4121C5B90
:01295E002256
:062FEF008E088F098D0A17
:102FF500908000E030E5079065787401F022906AD2
:10300500B4E0FCA3E0FDA3E0FEA3E0F5108E0F8D78
:103015000E8C0DE510FFE50F5407FEE42FF50CEEC1
:1030250034C0F50B850C82F5837423F0050CE50C93
:103035007002050B530BC7F582850B83EBF0050C6E
:10304500E50C7002050B530BC790633E63A2018527
:103055000B83850C8263A2017F06121F017406256E
:103065000CF50CE4350BF50B85088385098263A205
:1030750001850B83850C8263A201AF0A121F0174BF
:1030850008250AF50AFFE4FCFDFEE5102FF510EE14
:10309500350FF50FED350EF50EEC350DF50D908070
:1030A50040E50DF0A3E50EF0A3E50FF0A3E510F064
:1030B5009080007420F0AF10AE0FAD0EAC0D906A8D
:0430C500B4121C5BCA
:0130C90022E4
:02371D008F40DB
:10371F00908000E030E5079065787401F022906AA0
:10372F00B4E0FCA3E0FDA3E0FEA3E0F5448E438DDF
:10373F00428C41E544FFE5435407FEE42FFFEE348E
:10374F00C09062B463A201F5838F8263A201AF4080
:10375F00121F01E4FCFDFEE5442540F544EE354320
:10376F00F543ED3542F542EC3541F541908040E5AA
:10377F0041F0A3E542F0A3E543F0A3E544F09080C8
:10378F00007420F0AF44AE43AD42AC41906AB41226
:02379F001C5BB1
:0137A1002205
:062E32008E278F28AB057E
:102E3800908000E030E5079065787401F022906A90
:102E4800B4E0FCA3E0FDA3E0FEA3E0F52E8E2D8DFB
:102E58002C8C2BE52EFFE52D5407FEE42FF52AEEEA
:102E680034C0F529852A82F5837423F0052AE52ADA
:102E7800700205295329C7F582852983EBF0052AB5
:102E8800E52A7002052990633E63A201852983859E
:102E98002A8263A2017F06121F017406252AF52AD9
:102EA800E43529F5295329C7E527852A8285298309
:102EB800F0052AE52A700205295329C7F5828529D4
:102EC80083E528F0052AE52A700205295329C7E574
:102ED8002E240AF52EE4352DF52DE4352CF52CE4B9
:102EE800352BF52B908040E52BF0A3E52CF0A3E5DE
:102EF8002DF0A3E52EF09080007420F0AF2EAE2DBB
:0A2F0800AD2CAC2B906AB4121C5BD8
:012F1200229C
:10398C00908009E04480F09080E97441F07F0990C8
:10399C0080F6EFF0A37464F09080037402F09080D2
:1039AC0003E020E1F99069B0121C67000000009060
:1039BC0069B0E0908064F09069B1E0908065F0901F
:1039CC0069B2E0908066F09069B3E0908067F0A3F4
:1039DC00E4F0A3F0A3F0A3F090803CF0A3F0A3F0EC
:0239EC00A3F046
:0139EE0022B6
:102F13009081E9E0F52805280528052805280528D6
:102F230005280528052805280528908034E0F5297B
:102F3300A3E0F52AA3E0F52BA3E0F52C9081EAE0CA
:102F4300F528052805280528052805280528052826
:102F5300052805280528908038E0F52DA3E0F52EF7
:102F6300A3E0F52FA3E0F530E52FB52B08E530B549
:102F73002C037F0022AF30AE2FAD2EAC2DAB2CAA8D
:102F83002BA92AA829D3121C4A400AAF30AE2CEE33
:102F93009FF528800AAF30EFF404AE2C2EF528E518
:102FA3002F540744E0F58385308263A2019069B40E
:102FB30063A201AF28121F75E4FCFDFEE53025284E
:102FC300F530EE352FF52FED352EF52EEC352DF5AD
:102FD3002D908038E52DF0A3E52EF0A3E52FF0A387
:0B2FE300E530F09080037440F0AF2850
:012FEE0022C0
:022C5A008F28C1
:102C5C009080E8E0640660037FFF229069B0E0FC9E
:102C6C00A3E0FDA3E0FEA3E0F52C8E2B8D2A8C298E
:102C7C00E4FFFEFDFCAB2CAA2BA92AA829C3121C2D
:102C8C004A70609081F9E0F5299069B0E0FCA3E00E
:102C9C00FDA3E0FEA3E0FFE4FAF9F8EF2401FFEA5C
:102CAC003EFEE93DFDE83CFC9069B0121C5B90696E
:102CBC00B0E0FCA3E0FDA3E0FEA3E0FFE4F8EF240A
:102CCC0001FFEA3EFEE93DFDE83CFC9069B0121CB8
:102CDC005B908064E0F529A3E0F52AA3E0F52BA333
:102CEC00E0F52C9069B463A201E52B540744D8F5A8
:102CFC0083852C8263A201AF28121F2FE4FCFDFEFA
:102D0C00E52C2528F52CEE352BF52BED352AF52A5F
:102D1C00EC3529F529908064E529F0A3E52AF0A388
:102D2C00E52BF0A3E52CF09080037420F0AF2CAED3
:0D2D3C002BAD2AAC299069B0121C5B7F0002
:012D49002267
:0A3DB700E4FEEEC39F50030E80F8F7
:013DC10022DF
:103D0F00A2AF9227C2AF438E2075D2028F828E83CD
:0C3D1F00E0FFE4F5D2538EDFA22792AF44
:013D2B002275
:103CA300E5D220E0FBA2AF9227C2AF43D2028F82BC
:103CB3008E83EDF075D25063D250A22792AFE5D236
:033CC30020E0FB03
:013CC60022DB
:10382600E4FDED2401FFE433FE123D0F74362DF561
:1038360082E43463F583EFF00DBD3FE6E4FDED244D
:103846007FFFE433FE123D0F742D2DF582E43461C3
:10385600F583EFF0742D2DF582E43461F583E07085
:103866001B742D2DF582E43461F5837420F0742EDB
:103876002DF582E43461F583E4F080040DBD80BE4D
:10388600E49061ACF0FDEDFF7E00123D0F74AD2DAE
:0D389600F582E43461F583EFF00DBDFEE92D
:0138A3002202
:023C48008B2CC3
:103C4A00A2AF9227C2AF85A22D53A2FE8E838F8286
:103C5A0005A28C838D827409121F8BE52C53A2FE58
:103C6A0043A220121F8D53A2DF852DA2A22792AF55
:013C7A00FF4A
:013C7B002226
:103D2C00A2AF9227C2AF8C838D82EF121F8B43A25E
:0C3D3C0020121F8D53A2DFA22792AFFFC0
:013D48002258
:023CC7008F2745
:103CC900A2AF9227C2AFE4F5838D827406121F8BCF
:103CD900E52743A220121F8D53A2DFA22792AF7FAF
:013CE90001D9
:013CEA0022B7
:023CEB008F2721
:103CED00A2AF9227C2AFE4F5838D82740A121F8BA7
:103CFD00E52743A220121F8D53A2DFA22792AF7F8B
:013D0D0001B4
:013D0E002292
:101DB400A907E7FFA805EF93C3966008403B74FCAE
:101DC4002FFF80F00F08EF93C3966008402B74FB3D
:101DD4002FFF80E00F08EF93C3966008401B74FA4E
:101DE4002FFF80D00F08EF93D3966008400B74F94F
:101DF4002FFF80C01F1F1F1F1FEF54FEF80303F7A0
:101E0400E893FC08E893FD08E893FE08E893FF22B2
:101E140009E993C39D6008402974FB29F980F109FD
:101E2400E993C39E6008401A74FA29F980E209E92B
:101E340093D39F6008400B74F929F980D3191919B9
:101E44001919E9C313C313FF22740093F8ECC39860
:101E54004024701F740193F8EDC3984019701474F2
:0E1E64000293F8EEC398400E7009740393F8D1
:101E7200EFC39840037F00227F0122EDF8E6F008CD
:101E8200A3DFFA22EDF8E0F608A3DFFA22E0A3636B
:101E9200A201F0A363A201DFF475A2002263A201F2
:101EA200F0A363A20122E0A363A201F0A363A20153
:101EB200E0A363A201F0A363A201E463A201F0A381
:101EC20063A201DFE175A20022E0A363A2016DFE1D
:101ED200936CFDEE058393FC158363A201DFEA7523
:101EE200A200227F00E493A363A201F00F600CA37F
:101EF200E583C2E3F58363A20180EA75A20022E0D2
:101F0200A363A201F0A3E583C2E3F58363A201DF29
:101F1200EE75A20022E0A363A201F0A3E583C2E46E
:101F2200D2E3F58363A201DFEC75A20022E0A36392
:101F3200A201F0A3E58344F8C2E5F58363A201DFC1
:101F4200EC75A20022E583C2E3F583E0A363A2015C
:101F5200F0A363A201DFEE75A20022E583C2E4D200
:0A1F6200E3F583E0A363A201F0A3FE
:101F6C0063A201DFEC75A20022E58344F8F583E05F
:101F7C00A363A201F0A363A201DFEE75A20022F914
:101F8C0022C002C004C00612FFF0D006D004D0025A
:011F9C002222
:10350A00020869E493A3F8E493A34003F68001F266
:10351A0008DFF48029E493A3F85407240CC8C333C2
:10352A00C4540F4420C8834004F456800146F6DF91
:10353A00E4800B0102040810204080903D49E47E9B
:10354A00019360BCA3FF543F30E509541FFEE49386
:10355A00A360010ECF54C025E060A840B8E493A34D
:10356A00FAE493A3F8E493A3C8C582C8CAC583CA78
:10357A00F0A3C8C582C8CAC583CADFE9DEE780BE30
:013D6400005E
:101B4300BB010689828A83E0225002E722BBFE02A0
:091B5300E32289828A83E49322D3
:101B5C00BB010689828A83F0225002F722BBFE0168
:021B6C00F32262
:101B6E0075F008758200EF2FFFEE33FECD33CDCC2E
:101B7E0033CCC58233C5829BED9AEC99E5829840B1
:101B8E000CF582EE9BFEED9AFDEC99FC0FD5F0D68E
:101B9E00E4CEFBE4CDFAE4CCF9A88222B800C1B9B8
:101BAE000059BA002DEC8BF084CFCECDFCE5F0CBF6
:101BBE00F97818EF2FFFEE33FEED33FDEC33FCEB2F
:101BCE0033FB10D703994004EB99FB0FD8E5E4F9EA
:101BDE00FA227818EF2FFFEE33FEED33FDEC33FCD7
:101BEE00C933C910D7059BE99A4007EC9BFCE99ACB
:101BFE00F90FD8E0E4C9FAE4CCFB2275F010EF2F10
:101C0E00FFEE33FEED33FDCC33CCC833C810D7070F
:101C1E009BEC9AE899400AED9BFDEC9AFCE899F84A
:0E1C2E000FD5F0DAE4CDFBE4CCFAE4C8F922DD
:0E1C3C00C3E49FFFE49EFEE49DFDE49CFC22B9
:101C4A00EB9FF5F0EA9E42F0E99D42F0E89C45F0F0
:011C5A002267
:0C1C5B00ECF0A3EDF0A3EEF0A3EFF022FC
:101C6700A8828583F0D083D082121C7E121C7E123C
:101C77001C7E121C7EE473E493A3C583C5F0C58361
:101C8700C8C582C8F0A3C583C5F0C583C8C582C8C7
:011C9700222A
:1017E700E53B242FF8E6053B22782C302E02782F94
:1017F700E475F001121D14021B432027EB7F2ED244
:10180700278018EF540F2490D43440D4FF302B0B8B
:10181700EF24BFB41A0050032461FFE53C600215B2
:101827003C053FE53F7002053E302E0D782CE475F0
:10183700F001121D14EF021B5C023B597403D22EF8
:101847008003E4C22EF53B8B2C8A2D892EE4F53CD0
:10185700F53EF53FE53C60077F2012182280F575BD
:101867003DFFC228C227C229C22AC22CC22DC22FBD
:101877001217F0FF700D302E057F00121833AF3F9F
:10188700AE3E22B4255FC2D5C22B1217F0FF24D07B
:10189700B40A00501A75F00A783C30D50508B6FF2F
:1018A7000106C6A426F620D5047002D22A80D924C0
:1018B700CFB41A00EF5004C2E5D22B021A33D22854
:1018C70080C6D22780C0D22980BCD2D580BAD22C7C
:1018D70080B47F201218222029077401B53C0040EC
:1018E700F11217E7FF12182202185BD22FD22D80B0
:1018F700951217E7FB1217E7FA1217E7F94A4B7029
:101907000679047A1B7BFF20292EE53C602A7E009E
:101917008E82758300121C9860060EEE653D70F08E
:10192700C2D5EBC0E0EAC0E0E9C0E0EE121A7AD017
:10193700E0F9D0E0FAD0E0FB121B43FF60AAEBC04E
:10194700E0EAC0E0E9C0E0121822D0E02401F9D0B3
:10195700E03400FAD0E0FBE53D0460DCD53DD980FA
:10196700877BFF7A1A7976D229809C791080027951
:1019770008C22DC22F8008D2D5790A8004790AC2FD
:10198700D5E53D047002F53DE4FAFDFEFF1217E7C9
:10199700FC7B082028131217E7FD7B1030270A125B
:1019A70017E7FE1217E7FF7B20EC3382D592D5505D
:1019B70013C3E43027069FFFE49EFEE42028039D1F
:1019C700FDE49CFCE4CBF8C228EC700CCFCECDCC68
:1019D700E824F8F870F38017C3EF33FFEE33FEED1A
:1019E70033FDEC33FCEB33FB994002FB0FD8E9EBFB
:1019F700302805F8D0E0C448B228C0E00AEC4D4EC4
:101A07004F78207B0070C2EAB53D0040BCC0E012B1
:101A17001A7CD0F0D0E0202804C4C0E0C4B228C0AB
:101A2700F012180BD0F0D5F0EB02185B121D7318EB
:101A3700F85319725818C94C18C54219764F197EB0
:0F1A470044197E4918DE431984551968461968F9
:101A5600451968471B245018CD2D18D12E18F42B84
:101A660018D52318F2201B0D2A188D48000018ECF3
:101A76003F3F3F00790AA2D5202A14302C09B9101D
:101A8600020404B9080104A2D5202D025001042045
:101A960029689229B53C005034C0E07F20302A19CD
:101AA6007F30A229722D722C500F121AD3C229C26E
:101AB6002DC22CC22F7F30800F302C03E9C0E012DC
:101AC6001822302C03D0E0F9D0E0B53CCC302C17EE
:101AD6007F30B9100C1218227F58302B077F788080
:101AE60003B908031218223029057F2D0218227F18
:101AF60020202FF87F2B202DF322922980CF286ECD
:101B0600756C6C2900D2281217E73028F8C228789D
:101B16003C30D50108F602188D2D5043495812174E
:101B2600E72403B405004001E4901B1F9312181329
:0D1B3600743A121813D22A753C0402197279
:101F9D008B278A288929E4F533F532F531F530F5AB
:101FAD002EF52FE52B452C452A6012EBC0E0EAC03B
:101FBD00E0E9C0E0AB2AAA2BA92C121D24AB270502
:101FCD0029E529AA287002052814F9121B43F534B6
:101FDD00C394094007E534D3940D40E1E534642002
:101FED0060DBE534B42D05432F038016E534B42BA7
:101FFD0005432F01800C74FF2529F52974FF352821
:10200D00F528E52D60046410703FAB27AA28A92997
:10201D00121B4364306009E52D702E752D0A802941
:10202D00900001121C98FF64786004EFB4581343BC
:10203D002F01752D1074022529F529E43528F52871
:10204D008007E52D7003752D08AB270529E529AA15
:10205D00287002052814F9121B43F534C39461400E
:10206D000AE534D3947A50035334DF74D02534F514
:10207D0034C3940A400CE5349411406D74F9253441
:10208D00F534E534D3952D5060432F0185333885D4
:10209D003237853136853035AF2D7E00E4FCFDAB12
:1020AD0033AA32A931A830121CC5C8ECC8C9EDC974
:1020BD00CAEECACBEFCBE4FCFDFEEB2534F533EED7
:1020CD003AF532ED39F531EC38F530AF33AE32AD9E
:1020DD0031FCAB38AA37A936A835D3121C4A5003A8
:1020ED00022056432F04022056E52F20E003E48002
:1020FD002DE52B452C452A601EAB27E52924FFF93C
:10210D00E52834FFFAEBC0E0EAC0E0E9C0E0AB2A15
:10211D00AA2BA92C121D24E52F30E20774FFFFFE18
:10212D00FDFC22E52FAF33AE32AD31AC3030E103E3
:04213D00021C3C2222
:101C9800BB010CE58229F582E5833AF583E0225001
:101CA80006E92582F8E622BBFE06E92582F8E2224B
:0D1CB800E58229F582E5833AF583E4932265
:101CC500E88FF0A4CC8BF0A42CFCE98EF0A42CFCBE
:101CD5008AF0EDA42CFCEA8EF0A4CDA8F08BF0A43C
:101CE5002DCC3825F0FDE98FF0A42CCD35F0FCEB9B
:101CF5008EF0A4FEA9F0EB8FF0A4CFC5F02ECD3960
:0F1D0500FEE43CFCEAA42DCE35F0FDE43CFC22CC
:101D1400FAE6FB0808E6F925F0F618E6CA3AF622D0
:101D2400BB011A89828A83D0F0D0E0F8D0E0F9D0E0
:101D3400E0FAD0E0FBE8C0E0C0F0021DA25016E9D2
:101D4400F8D083D082D0E0F9D0E0FAD0E0FBC082B2
:101D5400C083021D99BBFE16E9F8D083D082D0E07F
:0F1D6400F9D0E0FAD0E0FBC082C083021DAB22B1
:101D7300D083D082F8E4937012740193700DA3A3FF
:101D830093F8740193F5828883E473740293686013
:061D9300EFA3A3A380DF13
:091D9900EBF608EAF608E9F6226F
:091DA200EBF0A3EAF0A3E9F02242
:091DAB00EBF208EAF208E9F22269
:00000001FF
